:100000003A288900831608148312080835288800C6
:100010008316081555308900AA308900881488187D
:100020000F28081135288F018E00FF308E07031C22
:100030008F07031C352803308D00DF302120152861
:100040008D01E83E8C008D09FC30031C2A288C07AA
:10005000031827288C0764008D0F27280C183028D8
:100060008C1C3428000034280800831303138312E7
:10007000640008008316C03086001F30850083129C
:1000800086108316861083120611831606118312BA
:100090008611831686118312061083160610C4304B
:1000A0008312132002308D0060302120B201A8019C
:1000B000A501A4012D10B301B401B5018121640093
:1000C000861B5E28B20A09308F00373014200130B9
:1000D0008D00283021203208B6003608083CB600D2
:1000E00064003608003C031D5E28B301B401B5016D
:1000F000061483160610831281216400051C7C28D7
:10010000C430132002308D006030212064000518B7
:100110008628A521B301B401B5012808B600360828
:100120000C3CB60064003608003C031D9A28A80168
:100130002D147C28B9212708B6003608013CB600EA
:1001400064003608003C031D7C282408B6003608ED
:10015000043CB60064003608003C031D3A298901BE
:1001600029080720013089002A0807200230890069
:100170002B080720033089002C080720A7012D1029
:10018000A80181216400051CC128C430132002305D
:100190008D006030212064000518CB28B301B40124
:1001A000B50104300120A600A60364002608003C27
:1001B00003194C28A5212808B6003608013CB600D2
:1001C00064003608003C031DE92886148316861057
:1001D00083122808B6003608023CB60064003608D0
:1001E000003C031DF728861083168610831228080A
:1001F000B6003608043CB60064003608003C031D17
:10020000052906158316061183122808B60036083C
:10021000053CB60064003608003C031D1329061196
:100220008316061183122808B6003608073CB6006C
:1002300064003608003C031D2129861583168611AB
:1002400083122808B6003608083CB6006400360859
:10025000003C031D2F29861183168611831228085E
:10026000B60036080B3CB60064003608003C0319A3
:100270004C28C02800300120AE0001300120AF0022
:1002800002300120B00003300120B1002908B6007F
:1002900036082E02B60064003608003C031D4C28C8
:1002A0002A08B60036082F02B60064003608003C63
:1002B000031D4C282B08B60036083002B600640037
:1002C0003608003C031D4C282C08B60036083102C5
:1002D000B60064003608003C031D4C28A701A801A5
:1002E0000430A40000302D180130B6003608013C5F
:1002F000B60064003608003C03197C28C02863005F
:100300007F29B30A3308B6003608FF3CB600640004
:100310003608003C03198D290800B40A3408B600D9
:100320003608FF3CB60064003608003C03199929E2
:100330000800B50A3508B6003608123CB60064005D
:100340003608003C03194C2808006400851CAA29C3
:100350000830A8076400051DAF290430A807640011
:10036000851DB4290230A8076400051EB829A80A13
:100370000800A50A2508B6003608013CB60064004E
:100380003608003C031DC8292808A900A801080058
:100390002508B6003608023CB60064003608003C6A
:1003A000031DD6292808AA00A80108002508B600C0
:1003B0003608033CB60064003608003C031DE429FF
:1003C0002808AB00A80108000130A7002808AC00ED
:0603D000A801A5010800D0
:02400E00F53F7C
:0A42000002000A000A0005000A008F
:00000001FF
